:1000000000308A00212800002B30840000080319EA
:1000100016280230A100A001A00B0C28A10B0B2870
:100020009730A000A00B1228800B092800342A0862
:1000300085003230AB00042085013230AB00042053
:10004000003484011F3083051F1383161F149F146F
:100050001F159F15073083129F00703083168F0085
:1000600070308F0007308312990083160508063020
:100070008312A000A00B3A28000019088C111F134E
:1000800083161F109F101F119F11083065008312E7
:10009000A6012608023C031C58283730850064302E
:1000A000AB00042085016430AB000420A60A492877
:1000B000851D5828A901A801851D69280330A000C5
:1000C000A00B6028000000000130A8070318A90A4F
:1000D0005C288501A91B7328A908031D7628280818
:1000E000793C031C762804308500D028A91B7F2882
:1000F000A908031D83282808833C031C8328043097
:10010000AA001720D028A91B8C28A908031D8F2816
:100110002808893C031C8F2802308500D028A91BA1
:100120009828A908031D9C282808943C031C9C2897
:100130000230AA001720D028A91BA528A908031D52
:10014000A82828089A3C031CA82801308500D0283C
:10015000A91BB128A908031DB5282808A43C031C25
:10016000B5282030AA001720D028A91BBE28A9082E
:10017000031DC1282808AB3C031CC1282030850082
:10018000D028A91BCA28A908031DCE282808B53CD9
:10019000031CCE281030AA001720D028103085006C
:0401A0005828630078
:02400E00C43CB0
:00000001FF
